:020000040800F2
:1000000000060020A10200088D1000080D10000855
:10001000651000080D10000839100008A302000840
:10002000A3020008A3020008A3020008CD290008CB
:10003000A3020008A3020008A3020008A30200080C
:10004000A3020008A3020008A3020008A3020008FC
:10005000A3020008A3020008553E0008813E0008E4
:10006000AD3E0008D93E0008053F0008A302000885
:10007000A3020008A3020008A3020008A3020008CC
:10008000A3020008A3020008A3020008A3020008BC
:10009000A3020008A3020008A3020008313F0008E1
:1000A000A3020008A3020008A3020008A30200089C
:1000B000A3020008A3020008A3020008A30200088C
:1000C000A3020008A3020008A3020008A30200087C
:1000D000A3020008A3020008A3020008A30200086C
:1000E000953F0008A3020008A3020008A30200082D
:1000F000A3020008A3020008A3020008A30200084C
:10010000A3020008A30200081D400008A302000883
:10011000A3020008A3020008A3020008A30200082B
:10012000A3020008A3020008A3020008A30200081B
:10013000A3020008A3020008A3020008A30200080B
:10014000A3020008A3020008A3020008A3020008FB
:10015000A3020008A3020008A3020008A3020008EB
:10016000A3020008A3020008A3020008A3020008DB
:10017000A302000839350008A3020008A302000802
:10018000A3020008A302000809400008A302000817
:10019000A3020008A3020008A3020008A3020008AB
:1001A000A3020008A3020008A3020008A30200089B
:1001B000A3020008A3020008A3020008A30200088B
:1001C000A3020008A3020008A3020008A30200087B
:1001D000A302000825350008A3020008A3020008B6
:1001E000A3020008A3020008A3020008A30200085B
:1001F000A3020008A3020008A3020008A30200084B
:10020000A3020008A3020008A3020008A30200083A
:10021000A3020008A3020008A3020008A30200082A
:10022000A3020008A3020008A3020008A30200081A
:10023000A3020008A3020008A3020008A30200080A
:10024000A3020008A3020008A3020008A3020008FA
:10025000A3020008A3020008A3020008A3020008EA
:10026000A3020008A3020008A3020008A3020008DA
:10027000A3020008A3020008A3020008A3020008CA
:10028000A3020008A3020008A3020008A3020008BA
:10029000A3020008A3020008A3020008A3020008AA
:1002A00002E000F000F8FEE73B48804772B63B48AA
:1002B00080F308883A4880F309883A484EF6085196
:1002C000CEF20001086040F20000CCF200004EF6D1
:1002D0003471CEF200010860BFF34F8FBFF36F8F10
:1002E00040F20000C0F2F0004EF68851CEF200015C
:1002F0000860BFF34F8FBFF36F8F4FF00000E1EE48
:10030000100A4EF63C71CEF200010860062080F320
:100310001488BFF36F8F02F017FC02F0B9FB03F0F3
:1003200053FB4FF0553020491C4A91423CBF41F8E5
:10033000040BFAE71D491A4A91423CBF41F8040BED
:10034000FAE71B491B4A1C4B9A423EBF51F8040B6B
:1003500042F8040BF8E700201849194A91423CBFC3
:1003600041F8040BFAE702F0D1FB03F0B1FB154CA6
:10037000154DAC4203DA54F8041B8847F9E700F046
:1003800043F8124C124DAC4203DA54F8041B884770
:10039000F9E702F0B9BB0000911000080006002048
:1003A00000220020000000080000002000060020BD
:1003B00030440008002200205C220020602200203F
:1003C000FC460020A0020008A0020008A0020008CD
:1003D000A00200082DE9F04F2DED108AC1F80CD0D5
:1003E000D0F80CD0BDEC108ABDE8F08F002383F369
:1003F00011882846A047002001F0C4FEFEE701F066
:100400003FFE00DFFEE7000038B500F0F7FC30B13A
:10041000164B00220E211A725A729972DA7202F089
:1004200089FA054602F0BCFA0446D0B9104B9D4249
:1004300019D001339D4241F2883512BF0446002590
:100440000124002002F080FA0CB100F079F800F0ED
:1004500083FD00F019FC284600F020F900F070F848
:10046000F9E70025EDE70546EBE700BF0022002095
:10047000010007B008B500F0D3FBA0F120035842FB
:10048000584108BD07B541F21203022101A8ADF899
:10049000043000F0E3FB03B05DF804FB38B5202323
:1004A00083F311881748C3680BB101F0F1FE0023F4
:1004B000154A4FF47A71134801F0AEFE002383F31E
:1004C0001188124C236813B12368013B23606368D1
:1004D00013B16368013B63600D4D2B7833B96368DA
:1004E0007BB9022000F0AAFC322363602B78032B37
:1004F00007D163682BB9022000F0A0FC4FF47A7397
:10050000636038BD602200209D0400087C23002029
:1005100074220020084B187003280CD8DFE800F084
:1005200008050208022000F07BBC022000F068BC35
:10053000024B00225A607047742200207C23002066
:10054000F8B5504B504A1C461968013100F09980AB
:1005500004339342F8D162684C4B9A4240F2918046
:100560004B4B9B6803F1006303F500339A4280F024
:100570008880002000F0A2FB0220FFF7CBFF454B54
:100580000021D3F8E820C3F8E810D3F81021C3F80D
:100590001011D3F81021D3F8EC20C3F8EC10D3F8E5
:1005A0001421C3F81411D3F81421D3F8F020C3F8A0
:1005B000F010D3F81821C3F81811D3F81821D3F884
:1005C000802042F00062C3F88020D3F8802022F01F
:1005D0000062C3F88020D3F88020D3F8802042F056
:1005E0000072C3F88020D3F8802022F00072C3F894
:1005F0008020D3F8803072B64FF0E023C3F8084D66
:10060000D4E90004BFF34F8FBFF36F8F224AC2F8C3
:100610008410BFF34F8F536923F480335361BFF3CA
:100620004F8FD2F8803043F6E076C3F3C905C3F3A9
:100630004E335B0103EA060C29464CEA8177013907
:10064000C2F87472F9D2203B13F1200FF2D1BFF33C
:100650004F8FBFF36F8FBFF34F8FBFF36F8F536910
:1006600023F4003353610023C2F85032BFF34F8F9D
:10067000BFF36F8F202383F31188854680F30888AA
:100680002047F8BD0000020820000208FFFF010813
:10069000002200200044025800ED00E02DE9F04F58
:1006A00093B0A84B2022FF2100900AA89D6800F07B
:1006B000FDFBA54A1378A3B90121A4481170C360BA
:1006C000202383F31188C3680BB101F0E1FD0023FF
:1006D0009F4A4FF47A719D4801F09EFD002383F3F9
:1006E0001188009B13B19B4B009A1A609A4A1378A9
:1006F000032B03D000231370964A53604FF0000A77
:10070000009CD3465646D146012000F089FB24B117
:10071000904B1B68002B00F00E82002000F080FA46
:100720000390039B002BF2DB012000F069FB039B8D
:10073000213B162BE8D801A252F823F099070008B4
:10074000C107000855080008090700080907000844
:1007500009070008DD080008AB0A0008C509000801
:10076000270A00084F0A0008750A00080907000850
:10077000870A000809070008F90A00083908000874
:10078000090700083D0B0008A50700083908000804
:1007900009070008270A00080220FFF76BFE00285F
:1007A00040F0F381009B022105A8BAF1000F08BFB9
:1007B0001C4641F21233ADF8143000F04FFAA3E7B3
:1007C0004FF47A7000F02CFA071EEBDB0220FFF7E3
:1007D00051FE0028E6D0013F052F00F2D881DFE866
:1007E00007F0030A0D1013360523042105A805930D
:1007F00000F034FA17E004215248F9E70421574881
:10080000F6E704215648F3E74FF01C08404608F18C
:10081000040800F055FA0421059005A800F01EFA1E
:10082000B8F12C0FF2D101204FF0000900FA07F7C0
:1008300047EA0B0B5FFA8BFB00F084FB26B10BF051
:100840000B030B2B08BF0024FFF71CFE5CE7042101
:100850004448CDE7002EA5D00BF00B030B2BA1D104
:100860000220FFF707FE074600289BD00120002644
:1008700000F024FA0220FFF74DFE5FFA86F84046AA
:1008800000F02CFA044688B14046013600F036FAF2
:100890000028F2D1BA46044641F21213022105A8FB
:1008A0003E46ADF8143000F0D9F92DE72546012079
:1008B000FFF730FE234B9B68AB4207D9284600F078
:1008C000FFF9013040F066810435F3E70025224B43
:1008D000BA463E461D701F4B5D60ADE7002E3FF4EB
:1008E00061AF0BF00B030B2B7FF45CAF0220FFF723
:1008F00011FE322000F094F9B0F10008FFF652AF7B
:1009000018F003077FF44EAF0E4A08EB0503926818
:1009100093423FF647AFB8F5807F3FF743AF124BA6
:10092000B845019322DD4FF47A7000F079F9039015
:10093000039A002AFFF636AF039A0137019B03F8AA
:10094000012BEDE700220020782300206022002008
:100950009D0400087C230020742200200422002033
:10096000082200200C22002078220020C820FFF757
:1009700081FD074600283FF415AF1F2D11D8C5F1A2
:1009800020020AAB25F0030084494245184428BFE1
:100990004246019200F064FA019AFF217F4800F07C
:1009A00085FA4FEAA803C8F387027C4928460193D9
:1009B00000F084FA064600283FF46EAF019B05EB79
:1009C000830539E70220FFF755FD00283FF4EAAE22
:1009D00000F0B0F900283FF4E5AE0027B846704BB0
:1009E0009B68BB4218D91F2F11D80A9B01330ED028
:1009F00027F0030312AA134453F8203C0593404602
:100A0000042205A9043700F061FB8046E7E7384679
:100A100000F056F90590F2E7CDF81480042105A8FE
:100A200000F01CF908E70023642104A8049300F0F7
:100A30000BF900287FF4B6AE0220FFF71BFD00285B
:100A40003FF4B0AE049800F06BF90590E6E70023A0
:100A5000642104A8049300F0F7F800287FF4A2AE04
:100A60000220FFF707FD00283FF49CAE049800F039
:100A700059F9EAE70220FFF7FDFC00283FF492AEA7
:100A800000F068F9E1E70220FFF7F4FC00283FF4EA
:100A900089AE05A9142000F063F9074604210490EB
:100AA00004A800F0DBF83946B9E7322000F0B8F8C6
:100AB000071EFFF677AEBB077FF474AE384A07EB2C
:100AC0000903926893423FF66DAE0220FFF7D2FC15
:100AD00000283FF467AE27F003074F44B9453FF4C1
:100AE000ABAE484609F1040900F0EAF8042105908C
:100AF00005A800F0B3F8F1E74FF47A70FFF7BAFCFD
:100B000000283FF44FAE00F015F9002844D00A9BAE
:100B100001330BD008220AA9002000F0CFF90028E9
:100B20003AD02022FF210AA800F0C0F9FFF7AAFC62
:100B30001C4801F02DFB13B0BDE8F08F002E3FF4F0
:100B400031AE0BF00B030B2B7FF42CAE0023642192
:100B500005A8059300F078F8074600287FF422AE38
:100B60000220FFF787FC804600283FF41BAEFFF70A
:100B700089FC41F2883001F00BFB059800F026FA61
:100B800046463C4600F0DEF9BEE5064654E64FF028
:100B9000000907E6BA467FE637467DE67822002060
:100BA00000220020A0860100F7B50C46184E4FF435
:100BB0007A71054602FB01F396F90020501C0BD117
:100BC0001448294601930268176A2246B8478442AE
:100BD000019B03D1002310E0002AF1D096F90020F8
:100BE000511C01D0012A0DD10B4829460268166A12
:100BF0002246B047844205D10123084A01201370E0
:100C000003B0F0BD4FF4FA7001F0C2FA0020F7E72C
:100C100010220020F0290020CC230020C82300202F
:100C2000002307B5024601210DF107008DF80730BA
:100C3000FFF7BAFF20B19DF8070003B05DF804FB91
:100C40004FF0FF30F9E700000A46042108B5FFF72E
:100C5000ABFF80F00100C0B2404208BD074B0A461E
:100C600030B41978064B53F82140014623682046DA
:100C7000DD69044BAC4630BC604700BFC823002090
:100C800010410008A086010070B50A4E00240A4DEC
:100C900001F028FD308028683388834208D901F0AC
:100CA0001DFD2B6804440133B4F5003F2B60F2D3E3
:100CB00070BD00BFCA2300208423002001F0F0BDD6
:100CC00000F1006000F500300068704700F100603E
:100CD000920000F5003001F067BD0000054B1A6876
:100CE000054B1B889B1A834202D9104401F0F6BCC5
:100CF0000020704784230020CA23002038B5074D08
:100D000004462868204401F0EFFC28B928682044F4
:100D1000BDE8384001F0FABC38BD00BF8423002094
:100D20000020704700F1FF5000F58F10D0F8000848
:100D300070470000064991F8243033B1002308229F
:100D4000086A81F82430FFF7C1BF0120704700BF57
:100D500088230020014B1868704700BF0010005C1A
:100D6000244BF0B51A680446234BC2F30B06120C51
:100D70001F885868BE4293F9085028D09F89BE4208
:100D800006D101200C2505FB0033586893F9085063
:100D900041F201039A421CD041F203039A421AD055
:100DA00042F201039A4218D042F203039A4208BF6A
:100DB0005625621E0B46441E0A4493420FD214F974
:100DC000016F581C6EB1034600F8016CF5E7002076
:100DD000D8E75A25EDE75925EBE75825E9E7184606
:100DE00005E02C2482421C7001D9981C5D70401AC9
:100DF000F0BD00BF0010005C1422002000207047EE
:100E0000022804D1054B4FF400029A617047012873
:100E1000FCD1024B4FF48002F7E700BF00080258F4
:100E2000022803D1044B80229A6170470128FCD12B
:100E3000014B4022F8E700BF00080258022805D104
:100E4000064A536983F08003536170470128FCD13F
:100E5000024A536983F04003F6E700BF00080258D6
:100E6000002310B5934203D0CC5CC4540133F9E79E
:100E700010BD0000013810B510F9013F3BB191F9E8
:100E800000409C4203D11AB10131013AF4E71AB192
:100E900091F90020981A10BD1046FCE7034602465F
:100EA000D01A12F9011B0029FAD1704702440346F7
:100EB000934202D003F8011BFAE770472DE9F8438B
:100EC0001F4D14460746884695F8242052BBDFF88C
:100ED00070909CB395F824302BB92022FF2148460E
:100EE0002F62FFF7E3FF95F824004146C0F10802A6
:100EF00005EB8000A24228BF2246D6B29200FFF73F
:100F0000AFFF95F82430A41B17441E449044E4B26C
:100F1000F6B2082E85F82460DBD1FFF70BFF00281E
:100F2000D7D108E02B6A03EB82038342CFD0FFF7CF
:100F300001FF0028CBD10020BDE8F8830120FBE7AA
:100F400088230020024B1A78024B1A70704700BFAA
:100F5000C82300201022002038B5164C164D20461C
:100F600000F018FC2946204600F040FC2D6813488C
:100F7000D5F89020D2F8043843F00203C2F80438C0
:100F800001F006F90E49284600F03EFDD5F8902004
:100F90000C48D2F804380C49A04223F00203C2F8EE
:100FA00004384FF4E1330B6003D0BDE8384000F063
:100FB0004FBB38BDF02900201842000840420F0006
:100FC00020420008CC230020B023002038B50B4B72
:100FD00004461A780A4B53F822500A4B9D420CD013
:100FE000094B002118221846FFF760FF04600146F4
:100FF0002846BDE8384000F02BBB38BDC823002090
:1010000010410008F0290020B023002000B59BB05B
:10101000EFF3098168226846FFF722FFEFF30583AB
:10102000044B9A6BDA6A9A6A9A6A9A6A9A6A9A6A14
:101030009B6AFEE700ED00E000B59BB0EFF309818D
:1010400068226846FFF70CFFEFF30583044B9A6BA9
:101050009A6A9A6A9A6A9A6A9A6A9B6AFEE700BFD3
:1010600000ED00E000B59BB0EFF30981682268460F
:10107000FFF7F6FEEFF30583034B5A6B9A6A9A6A01
:101080009A6A9A6A9B6AFEE700ED00E0FEE70000BC
:1010900000B595B0132101A801F092FC9DF84F30E6
:1010A0007BB10023132101A88DF84F3001F082FCA1
:1010B000054BD3F8002882F30888D3F80438984702
:1010C000FEE715B05DF804FB0090F01F30B50A4450
:1010D000084D91420DD011F8013B5840082340F3D0
:1010E0000004013B2C4013F0FF0384EA5000F6D1CA
:1010F000EFE730BD2083B8ED02684368114301601B
:1011000003B1184770470000024A136843F0C00358
:10111000136070470078004013B50E4C204600F075
:101120008BFA04F1140000234FF400720A49009472
:1011300000F04CF9094B4FF40072094904F13800F2
:10114000009400F0C5F9074A074BC4E9172302B021
:1011500010BD00BFCC230020382400200911000856
:10116000382600200078004000E1F505037C30B50A
:10117000244C002918BF0C46012B11D1224B984258
:101180000ED1224BD3F8E82042F08042C3F8E82089
:10119000D3F8102142F08042C3F81021D3F8103167
:1011A0002268036EC16D03EB52038466B3FBF2F356
:1011B0006268150442BF23F0070503F0070343EA02
:1011C0004503CB60A36843F040034B60E36843F002
:1011D00001038B6042F4967343F001030B604FF000
:1011E000FF330B62510505D512F0102205D0B2F184
:1011F000805F04D080F8643030BD7F23FAE73F235E
:10120000F8E700BF18410008CC2300200044025832
:101210002DE9F047C66D05463768F4692107346249
:1012200019D014F0080118BF8021E20748BF41F02F
:101230002001A3074FF0200348BF41F040016007A1
:1012400048BF41F4807183F31188281DFFF754FFD4
:10125000002383F31188E2050AD5202383F3118844
:101260004FF40071281DFFF747FF002383F3118817
:101270004FF020094FF0000A14F0200838D13B0647
:1012800016D54FF0200905F1380A200610D589F34C
:101290001188504600F050F9002836DA0821281D40
:1012A000FFF72AFF27F080033360002383F31188C0
:1012B000790614D5620612D5202383F31188D5E967
:1012C00013239A4208D12B6C33B127F04007102129
:1012D000281DFFF711FF3760002383F31188E30611
:1012E00018D5AA6E1369ABB15069BDE8F04718472D
:1012F00089F31188736A284695F86410194000F044
:10130000B5F98AF31188F469B6E7B06288F31188F9
:10131000F469BAE7BDE8F087F8B515468268044677
:101320000B46AA4200D28568A1692669761AB542A1
:101330000BD218462A46FFF793FDA3692B44A361FD
:101340002846A3685B1BA360F8BD0CD9AF1B1846E9
:101350003246FFF785FD3A46E1683044FFF780FDED
:10136000E3683B44EBE718462A46FFF779FDE3685C
:10137000E5E7000083689342F7B50446154600D2BE
:101380008568D4E90460361AB5420BD22A46FFF7C5
:1013900067FD63692B4463612846A3685B1BA360F8
:1013A00003B0F0BD0DD93246AF1B0191FFF758FDD8
:1013B00001993A46E0683144FFF752FDE3683B4447
:1013C000E9E72A46FFF74CFDE368E4E710B50A4475
:1013D0000024C361029B8460C16002610362C0E9B2
:1013E0000000C0E9051110BD08B5D0E905329342EF
:1013F00001D1826882B98268013282605A1C4261DE
:1014000019700021D0E904329A4224BFC3684361B5
:1014100000F0DAFE002008BD4FF0FF30FBE70000CF
:1014200070B5202304460E4683F31188A568A5B144
:10143000A368A269013BA360531CA36115782269CC
:10144000934224BFE368A361E3690BB12046984748
:10145000002383F31188284607E03146204600F038
:10146000A3FE0028E2DA85F3118870BD2DE9F74F5D
:1014700004460E4617469846D0F81C904FF0200AB6
:101480008AF311884FF0000B154665B12A463146A4
:101490002046FFF741FF034660B94146204600F071
:1014A00083FE0028F1D0002383F31188781B03B05A
:1014B000BDE8F08FB9F1000F03D001902046C84776
:1014C000019B8BF31188ED1A1E448AF31188DCE727
:1014D000C160C361009B82600362C0E905111144D1
:1014E000C0E9000001617047F8B504460D46164694
:1014F000202383F31188A768A7B1A368013BA360E9
:1015000063695A1C62611D70D4E904329A4224BF97
:10151000E3686361E3690BB120469847002080F3DC
:10152000118807E03146204600F03EFE0028E2DA4E
:1015300087F31188F8BD0000D0E9052310B59A4261
:1015400001D182687AB982680021013282605A1C16
:1015500082611C7803699A4224BFC368836100F0EA
:1015600033FE204610BD4FF0FF30FBE72DE9F74F6B
:1015700004460E4617469846D0F81C904FF0200AB5
:101580008AF311884FF0000B154665B12A463146A3
:101590002046FFF7EFFE034660B94146204600F0C3
:1015A00003FE0028F1D0002383F31188781B03B0D9
:1015B000BDE8F08FB9F1000F03D001902046C84775
:1015C000019B8BF31188ED1A1E448AF31188DCE726
:1015D000026843681143016003B118477047000077
:1015E0001430FFF743BF00004FF0FF331430FFF714
:1015F0003DBF00003830FFF7B9BF00004FF0FF33A8
:101600003830FFF7B3BF00001430FFF709BF000008
:101610004FF0FF311430FFF703BF00003830FFF701
:1016200063BF00004FF0FF323830FFF75DBF0000AE
:1016300000207047FFF770BD044B03600023436038
:10164000C0E9023301230374704700BF3041000832
:1016500010B52023044683F31188FFF787FD02238A
:101660002374002383F3118810BD000038B5C369CB
:1016700004460D461BB904210844FFF7A9FF29467B
:1016800004F11400FFF7B0FE002806DA201D4FF425
:101690008061BDE83840FFF79BBF38BD02684368F2
:1016A0001143016003B118477047000013B5406B48
:1016B00000F58054D4F8A4381A681178042914D19C
:1016C000017C022911D11979012312898B4013421F
:1016D0000BD101A94C3002F077F8D4F8A4480246A7
:1016E000019B2179206800F0DFF902B010BD0000F5
:1016F000143001F0F9BF00004FF0FF33143001F057
:10170000F3BF00004C3002F0CBB800004FF0FF33C5
:101710004C3002F0C5B80000143001F0C7BF000023
:101720004FF0FF31143001F0C1BF00004C3002F027
:1017300097B800004FF0FF324C3002F091B8000033
:101740000020704710B500F58054D4F8A4381A680A
:101750001178042917D1017C022914D15979012368
:1017600052898B4013420ED1143001F059FF0246CA
:1017700048B1D4F8A4484FF4407361792068BDE8BB
:10178000104000F07FB910BD406BFFF7DBBF0000D9
:10179000704700007FB5124B012504260446036004
:1017A0000023057400F1840243602946C0E9023336
:1017B0000C4B0290143001934FF44073009601F0EB
:1017C0000BFF094B04F69442294604F14C000294A5
:1017D000CDE900634FF4407301F0D2FF04B070BD57
:1017E0005841000889170008AD1600080A68202330
:1017F00083F311880B790B3342F823004B791333B1
:1018000042F823008B7913B10B3342F8230000F523
:101810008053C3F8A41802230374002383F31188B0
:101820007047000038B5037F044613B190F8543078
:10183000ABB90125201D0221FFF730FF04F1140090
:101840006FF00101257700F0CBFC04F14C0084F827
:1018500054506FF00101BDE8384000F0C1BC38BD04
:1018600010B5012104460430FFF718FF0023237749
:1018700084F8543010BD000038B5044600251430FB
:1018800001F0C2FE04F14C00257701F091FF201D0C
:1018900084F854500121FFF701FF2046BDE838408D
:1018A000FFF750BF90F8803003F06003202B06D183
:1018B00090F881200023212A03D81F2A06D800206F
:1018C0007047222AFBD1C0E91D3303E0034A426777
:1018D00007228267C3670120704700BF2C220020C7
:1018E00037B500F58055D5F8A4381A681178042961
:1018F0001AD1017C022917D11979012312898B4051
:10190000134211D100F14C04204602F011F858B1F5
:1019100001A9204601F058FFD5F8A4480246019BD2
:101920002179206800F0C0F803B030BD01F10B034D
:10193000F0B550F8236085B004460D46FEB1202373
:1019400083F3118804EB8507301D0821FFF7A6FEFD
:10195000FB6806F14C005B691B681BB1019001F04C
:1019600041FF019803A901F02FFF024648B1039BF4
:101970002946204600F098F8002383F3118805B02B
:10198000F0BDFB685A691268002AF5D01B8A013B3A
:101990001340F1D104F18002EAE70000133138B5B9
:1019A00050F82140ECB1202383F3118804F58053D3
:1019B000D3F8A4281368527903EB8203DB689B6990
:1019C0005D6845B104216018FFF768FE294604F1FF
:1019D000140001F02FFE2046FFF7B4FE002383F32E
:1019E000118838BD7047000001F022B90123402260
:1019F000002110B5044600F8303BFFF757FA0023EA
:101A0000C4E9013310BD000010B52023044683F360
:101A100011882422416000210C30FFF747FA20464C
:101A200001F028F902232370002383F3118810BDED
:101A300070B500EB8103054650690E461446DA6026
:101A400018B110220021FFF731FAA06918B1102255
:101A50000021FFF72BFA31462846BDE8704001F01F
:101A60001BBA000083682022002103F0011310B587
:101A7000044683601030FFF719FA2046BDE8104095
:101A800001F096BAF0B4012500EB810447898D403E
:101A9000E4683D43A469458123600023A26063603C
:101AA000F0BC01F0B3BA0000F0B4012500EB8104F2
:101AB00007898D40E4683D43646905812360002304
:101AC000A2606360F0BC01F029BB000070B5022386
:101AD00000250446242203702946C0F888500C30A3
:101AE00040F8045CFFF7E2F9204684F8705001F0FA
:101AF00067F963681B6823B129462046BDE870403A
:101B0000184770BD037880F88C3005230370436854
:101B10001B6810B504460BB1042198470023A3604D
:101B200010BD000090F88C20436802701B680BB158
:101B3000052118477047000070B590F870300446D2
:101B400013B1002380F8703004F18002204601F0C8
:101B500053FA63689B68B3B994F8803013F060055A
:101B600035D00021204601F0FDFC0021204601F087
:101B7000EDFC63681B6813B10621204698470623D5
:101B800084F8703070BD204698470028E4D0B4F83F
:101B90008630A26F9A4288BFA36794F98030A56F00
:101BA000002B4FF0200380F20381002D00F0F28023
:101BB000092284F8702083F3118800212046D4E99B
:101BC0001D23FFF771FF002383F31188DAE794F8F0
:101BD000812003F07F0343EA022340F20232934262
:101BE00000F0C58021D8B3F5807F48D00DD8012BF7
:101BF0003FD0022B00F09380002BB2D104F1880279
:101C000062670222A267E367C1E7B3F5817F00F054
:101C10009B80B3F5407FA4D194F88230012BA0D1F2
:101C2000B4F8883043F0020332E0B3F5006F4DD0D2
:101C300017D8B3F5A06F31D0A3F5C063012B90D8AE
:101C40006368204694F882205E6894F88310B4F8A4
:101C50008430B047002884D0436863670368A36773
:101C60001AE0B3F5106F36D040F6024293427FF48B
:101C700078AF5C4B63670223A3670023C3E794F844
:101C80008230012B7FF46DAFB4F8883023F002036B
:101C9000A4F88830C4E91D55E56778E7B4F88030CA
:101CA000B3F5A06F0ED194F88230204684F88A30C4
:101CB00001F0E4F863681B6813B1012120469847DE
:101CC000032323700023C4E91D339CE704F18B0335
:101CD00063670123C3E72378042B10D1202383F308
:101CE00011882046FFF7BEFE85F311880321636843
:101CF00084F88B5021701B680BB12046984794F8EC
:101D00008230002BDED084F88B300423237063688C
:101D10001B68002BD6D0022120469847D2E794F8C2
:101D2000843020461D0603F00F010AD501F056F954
:101D3000012804D002287FF414AF2B4B9AE72B4BD9
:101D400098E701F03DF9F3E794F88230002B7FF437
:101D500008AF94F8843013F00F01B3D01A06204670
:101D600002D501F017FCADE701F008FCAAE794F8F2
:101D70008230002B7FF4F5AE94F8843013F00F011D
:101D8000A0D01B06204602D501F0ECFB9AE701F03B
:101D9000DDFB97E7142284F8702083F311882B462B
:101DA0002A4629462046FFF76DFE85F31188E9E6AD
:101DB0005DB1152284F8702083F31188002120463C
:101DC000D4E91D23FFF75EFEFDE60B2284F87020A8
:101DD00083F311882B462A4629462046FFF764FEE6
:101DE000E3E700BF88410008804100088441000803
:101DF00038B590F870300446002B3ED0063BDAB27E
:101E00000F2A34D80F2B32D8DFE803F037313108EE
:101E1000223231313131313131313737856FB0F8DC
:101E200086309D4214D2C3681B8AB5FBF3F203FBD4
:101E300012556DB9202383F311882B462A46294673
:101E4000FFF732FE85F311880A2384F870300EE024
:101E5000142384F87030202383F311880023204654
:101E60001A461946FFF70EFE002383F3118838BD8A
:101E7000C36F03B198470023E7E70021204601F034
:101E800071FB0021204601F061FB63681B6813B100
:101E90000621204698470623D7E7000010B590F8A2
:101EA00070300446142B29D017D8062B05D001D842
:101EB0001BB110BD093B022BFBD80021204601F0CD
:101EC00051FB0021204601F041FB63681B6813B100
:101ED000062120469847062319E0152BE9D10B234C
:101EE00080F87030202383F3118800231A461946A6
:101EF000FFF7DAFD002383F31188DAE7C3689B69F3
:101F00005B68002BD5D1C36F03B19847002384F8D9
:101F10007030CEE7024B0022C3E900339A6070476D
:101F200038280020002382680374054B1B689968D9
:101F30009142FBD25A68036042601060586070475B
:101F40003828002008B5202383F31188037C032B55
:101F500005D0042B0DD02BB983F3118808BD43693C
:101F600000221A604FF0FF334361FFF7DBFF0023CD
:101F7000F2E7D0E9003213605A60F3E70023826889
:101F80000374054B1B6899689142FBD85A6803603B
:101F9000426010605860704738280020054B19696E
:101FA00008741868026853601A601861012303748A
:101FB000FEF710BA382800204B1C30B5044687B015
:101FC0000A4D10D02B6901A8094A00F025F92046D6
:101FD000FFF7E4FF049B13B101A800F059F92B6946
:101FE000586907B030BDFFF7D9FFF8E7382800205F
:101FF000451F000838B50C4D044641612B698168C6
:102000009A68914203D8BDE83840FFF78BBF184665
:10201000FFF7B4FF01232C61014623742046BDE87D
:102020003840FEF7D7B900BF38280020044B1A68A3
:102030001B6990689B68984294BF002001207047FC
:102040003828002010B5084C236820691A685460AD
:102050002260012223611A74FFF790FF0146206974
:10206000BDE81040FEF7B6B93828002008B5FFF7E4
:10207000DDFF18B1BDE80840FFF7E4BF08BD000070
:10208000FFF7E0BFFEE7000010B50C4CFFF742FF82
:1020900000F0B4F880220A49204600F03BF8012302
:1020A00044F8180C037400F0A1FC002383F311889A
:1020B00062B60448BDE8104000F04CB8602800202B
:1020C0008C4100089C41000800F01CB9EFF311801E
:1020D00020B9EFF30583202282F3118870470000B6
:1020E00010B530B9EFF30584C4F3080414B180F3DC
:1020F000118810BDFFF7BAFF84F31188F9E70000DB
:10210000034A516853685B1A9842FBD8704700BF76
:10211000001000E082600222028270478368A3F10F
:102120007C0243F80C2C026943F83C2C426943F8CA
:10213000382C074A43F81C2CC268A3F1180043F856
:10214000102C022203F8082C002203F8072C7047F9
:10215000ED03000810B5202383F31188FFF7DEFF9D
:1021600000210446FFF746FF002383F31188204631
:1021700010BD0000024B1B6958610F20FFF70EBF16
:1021800038280020202383F31188FFF7F3BF0000D5
:1021900008B50146202383F311880820FFF70CFFC0
:1021A000002383F3118808BD49B1064B42681B69BF
:1021B00018605A60136043600420FFF7FDBE4FF0C3
:1021C000FF307047382800200368984206D01A680C
:1021D0000260506018465961FFF7A4BE70470000C6
:1021E00038B504460D462068844200D138BD0368E6
:1021F00023605C604561FFF795FEF4E7054B4FF007
:10220000FF3103F11402C3E905220022C3E90712DA
:10221000704700BF3828002070B51C4E05460C469C
:10222000C0E9032301F0BAFB334653F8142F9A4256
:102230000DD130620A2C2CBF00190A302A60C5E982
:102240000124C6E90555BDE8704001F091BB316A33
:10225000431AE31838BF1C469368A34202D90819F1
:1022600001F096FB73699A6894420CD85A68AC6086
:102270002B606A6015609A685D60121B9A604FF06F
:10228000FF33F36170BDA41A1B68ECE73828002007
:1022900038B51B4C636998420DD08168D0E9003293
:1022A00013605A600022C2609A680A449A604FF034
:1022B000FF33E36138BD03682246002142F8143F32
:1022C00093425A60C16003D1BDE8384001F05ABB67
:1022D0009A688168256A0A449A6001F05FFB636925
:1022E000411B9A688A42E5D9AB181D1A206A092D4C
:1022F00098BF01F10A02BDE83840104401F048BB24
:10230000382800202DE9F041184C002704F114066C
:10231000656901F043FB236AAA68C11A8A4215D88D
:102320001344D5F80C802362D5E9003213605A605B
:102330006369EF60B34201D101F024FB87F3118898
:102340002869C047202383F31188E1E76169B1421E
:1023500009D013441B1ABDE8F0410A2B2CBFC0184A
:102360000A3001F015BBBDE8F08100BF382800201D
:1023700000207047FEE70000704700004FF0FF307C
:102380007047000002290CD0032904D00129074816
:1023900018BF00207047032A05D8054800EBC2008B
:1023A0007047044870470020704700BF7C42000817
:1023B0003C2200203042000870B59AB0054608461D
:1023C000144601A900F0C2F801A8FEF767FD431CFE
:1023D0000022C6B25B001046C5E900342370032317
:1023E000023404F8013C01ABD1B202348E4201D870
:1023F0001AB070BD13F8011B013204F8010C04F887
:10240000021CF1E708B5202383F311880348FFF786
:1024100067FA002383F3118808BD00BFF02900206C
:1024200090F8803003F01F02012A07D190F8812034
:102430000B2A03D10023C0E91D3315E003F060032C
:10244000202B08D1B0F884302BB990F88120212AB4
:1024500003D81F2A04D8FFF725BA222AEBD0FAE7BF
:10246000034A426707228267C3670120704700BFA3
:102470003322002007B5052917D8DFE801F0191627
:1024800003191920202383F31188104A0121019098
:10249000FFF7CEFA019802210D4AFFF7C9FA0D485D
:1024A000FFF7EAF9002383F3118803B05DF804FB1A
:1024B000202383F311880748FFF7B4F9F2E72023BC
:1024C00083F311880348FFF7CBF9EBE7D04100080D
:1024D000F4410008F029002038B50C4D0C4C2A4678
:1024E0000C4904F10800FFF767FF05F1CA0204F187
:1024F00010000949FFF760FF05F5CA7204F11800E2
:102500000649BDE83840FFF757BF00BFC84200206A
:102510003C220020B4410008BC410008C74100082B
:1025200070B5044608460D46FEF7B8FCC6B2204614
:10253000013403780BB9184670BD32462946FEF7C0
:1025400099FC0028F3D10120F6E700002DE9F84FAF
:1025500005460C46FEF7A2FC2A49C6B22846FFF7FC
:10256000DFFF08B10136F6B227492846FFF7D8FF4A
:1025700008B11036F6B2632E0DD8DFF88890DFF878
:1025800088A0224FDFF88CB0DFF88C802E7846B917
:102590002670BDE8F88F29462046BDE8F84F01F0C7
:1025A000A1BD252E2AD1072249462846FEF762FC06
:1025B00050B9D8F800300735083444F8083CD8F84A
:1025C000043044F8043CE1E7082251462846FEF76F
:1025D00051FC98B9A21C0E4B197802320909C95D49
:1025E00002F8041C13F8011B01F00F015B45C95DE3
:1025F00002F8031CF0D118340835C7E7013504F898
:10260000016BC3E79C420008C7410008AD420008C7
:1026100000E8F11F0CE8F11FA4420008BFF34F8F40
:10262000044B1A695107FCD1D3F810215207F8D195
:10263000704700BF0020005208B50D4B1B78ABB9A6
:10264000FFF7ECFF0B4BDA68D10704D50A4A5A6052
:1026500002F188325A60D3F80C21D20706D5064A17
:10266000C3F8042102F18832C3F8042108BD00BF79
:1026700026450020002000522301674508B5114B74
:102680001B78F3B9104B1A69510703D5DA6842F089
:102690004002DA60D3F81021520705D5D3F80C2197
:1026A00042F04002C3F80C21FFF7B8FF064BDA688E
:1026B00042F00102DA60D3F80C2142F00102C3F8C3
:1026C0000C2108BD26450020002000520F289ABF8B
:1026D00000F5806040040020704700004FF4003097
:1026E00070470000102070470F2808B50BD8FFF77F
:1026F000EDFF00F500330268013204D1043083425B
:10270000F9D1012008BD0020FCE700000F2870B5BA
:10271000054645D8FFF7DAFC224CFFF77FFF064657
:10272000FFF78AFF4FF0FF33072D6361C4F81431C0
:1027300020D82361FFF772FF2B0243F02403E360EC
:10274000E36843F08003E36023695A07FCD428461A
:10275000FFF764FF4FF40031FFF7B8FF00F002F914
:102760003046FFF78BFFFFF7BBFC2846BDE8704003
:10277000FFF7BABFC4F81031FFF750FFA5F1080307
:102780001B0243F02403C4F80C31D4F80C3143F09D
:102790008003C4F80C31D4F810315B07FBD4D6E7C2
:1027A000002070BD002000522DE9F84F40EA0203DE
:1027B00005460C461746D80602D00020BDE8F88F23
:1027C00027F01F07DFF8D4B0FFF736FF2744BC42DD
:1027D00003D10120FFF752FFF0E7202229462046CF
:1027E00001F070FC10B920352034F0E72B4605F1DC
:1027F00020021E68711CE0D104339A42F9D1FFF720
:1028000065FC05F17843234AB3F5801F224B28BFAE
:102810009A4603F1040338BF9046A2F1080228BF8C
:102820009846A3F108033ABF9146DA469946FFF766
:10283000F5FEC8F80060A5EB040CD9F8002004F1FF
:102840001C0142F00202C9F80020221FDAF80060E1
:1028500016F00506FAD152F8043F8A424CF80230CD
:10286000F4D1BFF34F8FFFF7D9FE4FF0FF32C8F816
:102870000020D9F8002022F00202C9F80020FFF75A
:102880002FFC20222146284601F01CFC0028AAD05B
:1028900030469FE7142000521021005210200052B1
:1028A00010B5084C237828B11BB9FFF7C5FE0123EA
:1028B000237010BD002BFCD02070BDE81040FFF746
:1028C000DDBE00BF264500200244074BD2B210B542
:1028D000904200D110BD441C00B253F8200041F8D2
:1028E000040BE0B2F4E700BF504000580E4B30B587
:1028F0001C6F240405D41C6F1C671C6F44F4004437
:102900001C670A4C02442368D2B243F480732360EC
:10291000074B904200D130BD441C51F8045B00B21B
:1029200043F82050E0B2F4E700440258004802584F
:102930005040005807B5012201A90020FFF7C4FF4D
:10294000019803B05DF804FB13B50446FFF7F2FFEE
:10295000A04205D0012201A900200194FFF7C6FF83
:1029600002B010BD0144BFF34F8F064B884204D321
:10297000BFF34F8FBFF36F8F7047C3F85C022030F7
:10298000F4E700BF00ED00E0034B1A681AB9034AF0
:10299000D2F8D0241A607047284500200040025821
:1029A00008B5FFF7F1FF024B1868C0F3806008BD5F
:1029B00028450020CAB201460120FFF797BF00005A
:1029C000CAB201460120FFF77FBF0000EFF3098381
:1029D000054968334A6B22F001024A6383F3098890
:1029E000002383F31188704700EF00E0202080F37C
:1029F000118862B60D4B0E4AD96821F4E0610904D2
:102A0000090C0A430B49DA60D3F8FC2042F08072CB
:102A1000C3F8FC20084AC2F8B01F116841F0010158
:102A200011601022DA7783F82200704700ED00E091
:102A30000003FA0555CEACC5001000E0202310B508
:102A400083F311880E4B5B6813F4006314D0F1EE2E
:102A5000103AEFF309844FF08073683CE361094B4F
:102A6000DB6B236684F30988FFF7E0FA10B1064BAD
:102A7000A36110BD054BFBE783F31188F9E700BFA5
:102A800000ED00E000EF00E0FF0300080204000892
:102A900070B5BFF34F8FBFF36F8F1A4A0021C2F892
:102AA0005012BFF34F8FBFF36F8F536943F400335E
:102AB0005361BFF34F8FBFF36F8FC2F88410BFF322
:102AC0004F8FD2F8803043F6E074C3F3C900C3F3EC
:102AD0004E335B0103EA0406014646EA817501397B
:102AE000C2F86052F9D2203B13F1200FF2D1BFF3AC
:102AF0004F8F536943F480335361BFF34F8FBFF35C
:102B00006F8F70BD00ED00E0FEE700000A4B0B4840
:102B10000B4A90420BD30B4BC11EDA1C121A22F047
:102B200003028B4238BF00220021FEF7BFB953F8E1
:102B3000041B40F8041BECE78C440008FC46002012
:102B4000FC460020FC4600207047000070B5D0E92C
:102B5000244300224FF0FF359E6804EB42135101DD
:102B6000D3F80009002805DAD3F8000940F08040C6
:102B7000C3F80009D3F8000B002805DAD3F8000BDE
:102B800040F08040C3F8000B013263189642C3F84E
:102B90000859C3F8085BE0D24FF00113C4F81C38A1
:102BA00070BD000000EB8103D3F80CC02DE9F043A9
:102BB000DCF814204E1CD0F89050D2F800E005EB61
:102BC000063605EB4118506870450AD30122D5F846
:102BD000343802FA01F123EA0101C5F83418BDE8DE
:102BE000F083AEEB0003BCF81040A34228BF23469D
:102BF000D8F81849A4B2B3EB840FF0D89468A4F1C4
:102C0000040959F8047F3760A4EB09071F44042F17
:102C1000F7D81C44034494605360D4E7890141F021
:102C20002001016103699B06FCD41220FFF768BAFA
:102C300010B50A4C2046FEF7D9FE094BC4F8903077
:102C4000084BC4F89430084C2046FEF7CFFE074BE3
:102C5000C4F89030064BC4F8943010BD2C450020C9
:102C600000000840E4420008C8450020000004407D
:102C7000F042000870B503780546012B5DD1494B41
:102C8000D0F89040984259D1474B0E216520D3F897
:102C9000D82042F00062C3F8D820D3F8002142F0D7
:102CA0000062C3F80021D3F80021D3F8802042F05D
:102CB0000062C3F88020D3F8802022F00062C3F8BD
:102CC0008020D3F8803000F071FC384BE360384B43
:102CD000C4F800380023D5F89060C4F8003EC02343
:102CE00023604FF40413A3633369002BFCDA012340
:102CF0000C203361FFF704FA3369DB07FCD41220A0
:102D0000FFF7FEF93369002BFCDA00262846A6609F
:102D1000FFF71CFF6B68C4F81068DB68C4F8146820
:102D2000C4F81C68002B3AD1224BA3614FF0FF334B
:102D30006361A36843F00103A36070BD1E4B98421A
:102D4000C8D1194B0E214D20D3F8D82042F0007283
:102D5000C3F8D820D3F8002142F00072C3F8002154
:102D6000D3F80021D3F8802042F00072C3F880200D
:102D7000D3F8802022F00072C3F88020D3F880209E
:102D8000D3F8D82022F08062C3F8D820D3F80021ED
:102D900022F08062C3F80021D3F8003193E7074B9B
:102DA000C3E700BF2C4500200044025840140040F7
:102DB00003002002003C30C0C8450020083C30C061
:102DC000F8B5D0F89040054600214FF00066204647
:102DD000FFF724FFD5F8941000234FF001128F68FD
:102DE0004FF0FF30C4F83438C4F81C2804EB431209
:102DF00001339F42C2F80069C2F8006BC2F80809AB
:102E0000C2F8080BF2D20B68D5F89020C5F89830BC
:102E1000636210231361166916F01006FBD11220AD
:102E2000FFF76EF9D4F8003823F4FE63C4F80038D5
:102E3000A36943F4402343F01003A3610923C4F8BA
:102E40001038C4F814380B4BEB604FF0C043C4F893
:102E5000103B094BC4F8003BC4F81069C4F80039B2
:102E6000D5F8983003F1100243F48013C5F8982088
:102E7000A362F8BDC042000840800010D0F8902046
:102E800090F88A10D2F8003823F4FE6343EA011365
:102E9000C2F80038704700002DE9F84300EB8103C9
:102EA000D0F890500C468046DA680FFA81F9480154
:102EB000166806F00306731E022B05EB41134FF054
:102EC000000194BFB604384EC3F8101B4FF0010147
:102ED00004F1100398BF06F1805601FA03F39169DB
:102EE00098BF06F5004600293AD0578A04F15801E8
:102EF000374349016F50D5F81C180B430021C5F822
:102F00001C382B180127C3F81019A7405369611EFC
:102F10009BB3138A928B9B08012A88BF5343D8F82E
:102F20009820981842EA034301F140022146C8F86C
:102F30009800284605EB82025360FFF76FFE08EB0E
:102F40008900C3681B8A43EA845348341E436401E2
:102F50002E51D5F81C381F43C5F81C78BDE8F883FE
:102F600005EB4917D7F8001B21F40041C7F8001BF7
:102F7000D5F81C1821EA0303C0E704F13F030B4A0C
:102F80002846214605EB83035A60FFF747FE05EB11
:102F90004910D0F8003923F40043C0F80039D5F8BF
:102FA0001C3823EA0707D7E700800010000400025E
:102FB000D0F894201268C0F89820FFF7C7BD000031
:102FC0005831D0F8903049015B5813F4004004D0D8
:102FD00013F4001F0CBF0220012070474831D0F8C5
:102FE000903049015B5813F4004004D013F4001FE3
:102FF0000CBF02200120704700EB8101CB68196AE9
:103000000B6813604B6853607047000000EB81034E
:1030100030B5DD68AA691368D36019B9402B84BF45
:10302000402313606B8A1468D0F890201C4402EB94
:103030004110013C09B2B4FBF3F46343033323F0C2
:10304000030343EAC44343F0C043C0F8103B2B687A
:1030500003F00303012B0ED1D2F8083802EB411024
:1030600013F4807FD0F8003B14BF43F0805343F04B
:103070000053C0F8003B02EB4112D2F8003B43F092
:103080000443C2F8003B30BD2DE9F041D0F8906018
:1030900005460C4606EB4113D3F8087B3A07C3F804
:1030A000087B08D5D6F814381B0704D500EB81033C
:1030B000DB685B689847FA071FD5D6F81438DB073A
:1030C0001BD505EB8403D968CCB98B69488A5A684B
:1030D000B2FBF0F600FB16228AB91868DA68904253
:1030E0000DD2121AC3E90024202383F3118821464C
:1030F0002846FFF78BFF84F31188BDE8F081012398
:1031000003FA04F26B8923EA02036B81CB68002B7C
:10311000F3D021462846BDE8F041184700EB810373
:103120004A0170B5DD68D0F890306C692668E660B9
:1031300056BB1A444FF40020C2F810092A6802F066
:103140000302012A0AB20ED1D3F8080803EB421495
:1031500010F4807FD4F8000914BF40F0805040F094
:103160000050C4F8000903EB4212D2F8000940F005
:103170000440C2F800090122D3F8340802FA01F130
:103180000143C3F8341870BD19B9402E84BF4020E4
:10319000206020681A442E8A8419013CB4FBF6F49E
:1031A00040EAC44040F00050C6E700002DE9F0417D
:1031B000D0F8906004460D4606EB4113D3F8087929
:1031C000C3F80879FB071CD5D6F81038DA0718D5EC
:1031D00000EB8103D3F80CC0DCF81430D3F800E026
:1031E000DA6896451BD2A2EB0E024FF000081A6077
:1031F000C3F80480202383F31188FFF78FFF88F33F
:1032000011883B0618D50123D6F83428AB40134269
:1032100012D029462046BDE8F041FFF7C3BC012388
:1032200003FA01F2038923EA02030381DCF8083080
:10323000002BE6D09847E4E7BDE8F0812DE9F84F90
:10324000D0F8905004466E69AB691E4016F4805861
:103250006E6103D0BDE8F84FFEF738BC002E12DADD
:10326000D5F8003E9F0705D0D5F8003E23F00303B4
:10327000C5F8003ED5F80438204623F00103C5F810
:103280000438FEF74FFC300505D52046FFF75EFCFD
:103290002046FEF737FCB1040CD5D5F8083813F0FA
:1032A000060FEB6823F470530CBF43F4105343F440
:1032B000A053EB60320704D56368DB680BB120468E
:1032C0009847F30200F1BA80B70226D5D4F890905F
:1032D00000274FF0010A09EB4712D2F8003B03F434
:1032E0004023B3F5802F11D1D2F8003B002B0DDA2B
:1032F00062890AFA07F322EA0303638104EB870376
:10330000DB68DB6813B13946204698470137D4F8AB
:103310009430FFB29B689F42DDD9F00619D5D4F8EE
:103320009000026AC2F30A1702F00F0302F4F012CF
:10333000B2F5802F00F0CC80B2F5402F09D104EB1C
:103340008303002200F58050DB681B6A974240F03F
:10335000B2803003D5F8185835D5E90303D50021DC
:103360002046FFF791FEAA0303D501212046FFF76F
:103370008BFE6B0303D502212046FFF785FE2F034A
:1033800003D503212046FFF77FFEE80203D5042181
:103390002046FFF779FEA90203D505212046FFF755
:1033A00073FE6A0203D506212046FFF76DFE2B024D
:1033B00003D507212046FFF767FEEF0103D508215B
:1033C0002046FFF761FE700340F1A980E90703D5AD
:1033D00000212046FFF7EAFEAA0703D50121204677
:1033E000FFF7E4FE6B0703D502212046FFF7DEFE60
:1033F0002F0703D503212046FFF7D8FEEE0603D59D
:1034000004212046FFF7D2FEA80603D50521204659
:10341000FFF7CCFE690603D506212046FFF7C6FE5E
:103420002A0603D507212046FFF7C0FEEB0576D517
:1034300020460821BDE8F84FFFF7B8BED4F89090B9
:1034400000274FF0010AD4F894305FFA87FB9B689D
:103450009B453FF639AF09EB4B13D3F8002902F433
:103460004022B2F5802F24D1D3F80029002A20DA97
:10347000D3F8002942F09042C3F80029D3F800297C
:10348000002AFBDB5946D4F89000FFF7C7FB2289DE
:103490000AFA0BF322EA0303238104EB8B03DB68B4
:1034A0009B6813B159462046984759462046FFF776
:1034B00079FB0137C7E7910701D1D0F80080072ACF
:1034C00002F101029CBF03F8018B4FEA18283DE787
:1034D00004EB830300F58050DA68D2F818C0DCF8FA
:1034E0000820DCE9001CA1EB0C0C00218F4208D164
:1034F000DB689B699A683A449A605A683A445A6011
:1035000027E711F0030F01D1D0F800808C4501F1BD
:10351000010184BF02F8018B4FEA1828E6E7BDE8F5
:10352000F88F000008B50348FFF788FEBDE80840A3
:10353000FFF784BA2C45002008B50348FFF77EFE4C
:10354000BDE80840FFF77ABAC8450020D0F89030AF
:1035500003EB4111D1F8003B43F40013C1F8003BE9
:1035600070470000D0F8903003EB4111D1F80039DA
:1035700043F40013C1F8003970470000D0F89030D0
:1035800003EB4111D1F8003B23F40013C1F8003BD9
:1035900070470000D0F8903003EB4111D1F80039AA
:1035A00023F40013C1F8003970470000090100F14D
:1035B0006043012203F56143C9B283F8001300F0B0
:1035C0001F039A4043099B0003F1604303F56143E5
:1035D000C3F880211A60704730B50433039C017230
:1035E000002104FB0325C160C0E90653049B03636B
:1035F000059BC0E90000C0E90422C0E90842C0E917
:103600000A11436330BD00000022416AC260C0E974
:103610000411C0E90A226FF00101FEF7E1BD0000CC
:10362000D0E90432934201D1C2680AB9181D70472B
:1036300000207047036919600021C2680132C2602E
:10364000C269134482699342036124BF436A0361E0
:10365000FEF7BABD38B504460D46E3683BB1626972
:103660000020131D1268A3621344E36207E0237A6B
:1036700033B929462046FEF797FD0028EDDA38BD1C
:103680006FF00100FBE70000C368C269013BC36043
:103690004369134482699342436124BF436A43618F
:1036A00000238362036B03B11847704770B5202372
:1036B000044683F31188866A3EB9FFF7CBFF0546BF
:1036C00018B186F31188284670BDA36AE26A13F820
:1036D000015B9342A36202D32046FFF7D5FF00238C
:1036E00083F31188EFE700002DE9F84F04460E46FA
:1036F000174698464FF0200989F311880025AA46FD
:10370000D4F828B0BBF1000F09D141462046FFF79D
:10371000A1FF20B18BF311882846BDE8F88FD4E9CA
:103720000A12A7EB050B521A934528BF9346BBF12B
:10373000400F1BD9334601F1400251F8040B91426E
:1037400043F8040BF9D1A36A403640354033A362F5
:10375000D4E90A239A4202D32046FFF795FF8AF361
:103760001188BD42D8D289F31188C9E730465A463C
:10377000FDF776FBA36A5E445D445B44A362E7E722
:1037800010B5029C0433017204FB0321C460C0E93C
:1037900006130023C0E90A33039B0363049BC0E9BB
:1037A0000000C0E90422C0E90842436310BD0000E4
:1037B000026A6FF00101C260426AC0E9042200227D
:1037C000C0E90A22FEF70CBDD0E904239A4201D1D8
:1037D000C26822B9184650F8043B0B6070470020BD
:1037E00070470000C3680021C2690133C3604369A8
:1037F000134482699342436124BF436A4361FEF7E5
:10380000E3BC000038B504460D46E3683BB12369CC
:1038100000201A1DA262E2691344E36207E0237AE2
:1038200033B929462046FEF7BFFC0028EDDA38BD43
:103830006FF00100FBE7000003691960C268013AFC
:10384000C260C269134482699342036124BF436A20
:10385000036100238362036B03B1184770470000C4
:1038600070B520230D460446114683F31188866AFD
:103870002EB9FFF7C7FF10B186F3118870BDA36A98
:103880001D70A36AE26A01339342A36204D3E16923
:1038900020460439FFF7D0FF002080F31188EDE7C0
:1038A0002DE9F84F04460D46904699464FF0200A00
:1038B0008AF311880026B346A76A4FB949462046C5
:1038C000FFF7A0FF20B187F311883046BDE8F88FDD
:1038D000D4E90A073A1AA8EB0607974228BF174609
:1038E000402F1BD905F1400355F8042B9D4240F8A9
:1038F000042BF9D1A36A40364033A362D4E90A23EA
:103900009A4204D3E16920460439FFF795FF8BF30F
:1039100011884645D9D28AF31188CDE729463A461F
:10392000FDF79EFAA36A3D443E443B44A362E5E7AB
:10393000D0E904239A4217D1C3689BB1836A8BB143
:10394000043B9B1A0ED01360C368013BC360C3697C
:103950001A4483699A42026124BF436A03610023C7
:1039600083620123184670470023FBE700F0DAB8B2
:10397000034B002258631A610222DA60704700BFCD
:10398000000C0040014B0022DA607047000C004040
:10399000014B5863704700BF000C0040014B586A50
:1039A000704700BF000C00404B6843608B68836029
:1039B000CB68C3600B6943614B6903628B694362E7
:1039C0000B6803607047000008B53C4B40F2FF7184
:1039D0003B48D3F888200A43C3F88820D3F88820CE
:1039E00022F4FF6222F00702C3F88820D3F888206F
:1039F000D3F8E0200A43C3F8E020D3F808210A43B3
:103A0000C3F808212F4AD3F808311146FFF7CCFF3D
:103A100000F5806002F11C01FFF7C6FF00F5806031
:103A200002F13801FFF7C0FF00F5806002F1540198
:103A3000FFF7BAFF00F5806002F17001FFF7B4FFF5
:103A400000F5806002F18C01FFF7AEFF00F58060A9
:103A500002F1A801FFF7A8FF00F5806002F1C401A0
:103A6000FFF7A2FF00F5806002F1E001FFF79CFF85
:103A700000F5806002F1FC01FFF796FF02F58C7102
:103A800000F58060FFF790FF00F000F90E4BD3F8CF
:103A9000902242F00102C3F89022D3F8942242F01F
:103AA0000102C3F894220522C3F898204FF0605217
:103AB000C3F89C20054AC3F8A02008BD0044025862
:103AC00000000258FC42000800ED00E01F0008035F
:103AD00008B500F0D7FAFEF7D7FA0F4BD3F8DC2081
:103AE00042F04002C3F8DC20D3F8042122F0400267
:103AF000C3F80421D3F80431084B1A6842F00802D5
:103B00001A601A6842F004021A60FEF73DFFBDE831
:103B10000840FEF7E1BC00BF00440258001802480C
:103B200070470000114BD3F8E82042F00802C3F8B8
:103B3000E820D3F8102142F00802C3F810210C4A03
:103B4000D3F81031D36B43F00803D363C722094B7A
:103B50009A624FF0FF32DA6200229A615A63DA60A9
:103B60005A6001225A611A60704700BF004402582F
:103B70000010005C000C0040094A08B51169D368C8
:103B80000B40D9B29B076FEA0101116107D52023D1
:103B900083F31188FEF798FA002383F3118808BD98
:103BA000000C0040384B4FF0FF31D3F88020C3F8B1
:103BB0008010D3F880200022C3F88020D3F8800042
:103BC000D3F88400C3F88410D3F88400C3F88420A9
:103BD000D3F88400D86F40F0FF4040F4FF0040F479
:103BE0003F5040F03F00D867D86F20F0FF4020F4EE
:103BF000FF0020F43F5020F03F00D867D86FD3F883
:103C000088006FEA40506FEA5050C3F88800D3F83C
:103C10008800C0F30A00C3F88800D3F88800D3F8FE
:103C20009000C3F89010D3F89000C3F89020D3F818
:103C30009000D3F89400C3F89410D3F89400C3F81C
:103C40009420D3F89400D3F89800C3F89810D3F8D0
:103C50009800C3F89820D3F89800D3F88C00C3F8E4
:103C60008C10D3F88C00C3F88C20D3F88C00D3F8D8
:103C70009C00C3F89C10D3F89C10C3F89C20D3F888
:103C80009C3000F0D3B900BF00440258614B0122C0
:103C9000C3F80821604BD3F8F42042F00202C3F8C5
:103CA000F420D3F81C2142F00202C3F81C210222A6
:103CB000D3F81C31594BDA605A689104FCD5584A44
:103CC0001A6001229A60574ADA6000221A614FF4A2
:103CD00040429A61514B9A699204FCD51A6842F4A9
:103CE00080721A604C4B1A6F12F4407F04D04FF46C
:103CF00080321A6700221A671A6842F001021A60BD
:103D0000454B1A685007FCD500221A611A6912F057
:103D10003802FBD1012119604FF0804159605A6788
:103D2000414ADA62414A1A611A6842F480321A60E2
:103D3000394B1A689103FCD51A6842F480521A6014
:103D40001A689204FCD53A4A3A499A6200225A63A8
:103D500019633949DA6399635A64384A1A64384AEC
:103D6000DA621A6842F0A8521A602B4B1A6802F005
:103D70002852B2F1285FF9D148229A614FF4886243
:103D8000DA6140221A622F4ADA644FF080521A65D3
:103D90002D4A5A652D4A9A6532232D4A13601368BD
:103DA00003F00F03022BFAD11B4B1A6942F00302F6
:103DB0001A611A6902F03802182AFAD1D3F8DC2005
:103DC00042F00052C3F8DC20D3F8042142F0005244
:103DD000C3F80421D3F80421D3F8DC2042F0804258
:103DE000C3F8DC20D3F8042142F08042C3F8042158
:103DF000D3F80421D3F8DC2042F00042C3F8DC20E1
:103E0000D3F8042142F00042C3F80421D3F804316E
:103E1000704700BF0080005100440258004802581B
:103E200000C000F0020000010000FF0100889008BF
:103E300022204000630209012C0204004704050807
:103E4000FD0BFF01200000200010E0000001010038
:103E5000002000524FF0B04208B5D2F8883003F08D
:103E60000103C2F8883023B1044A13680BB15068CB
:103E70009847BDE80840FEF7E1BD00BF7C46002042
:103E80004FF0B04208B5D2F8883003F00203C2F810
:103E9000883023B1044A93680BB1D0689847BDE8D5
:103EA0000840FEF7CBBD00BF7C4600204FF0B0427B
:103EB00008B5D2F8883003F00403C2F8883023B183
:103EC000044A13690BB150699847BDE80840FEF7F2
:103ED000B5BD00BF7C4600204FF0B04208B5D2F817
:103EE000883003F00803C2F8883023B1044A93698C
:103EF0000BB1D0699847BDE80840FEF79FBD00BFF1
:103F00007C4600204FF0B04208B5D2F8883003F06C
:103F10001003C2F8883023B1044A136A0BB1506A07
:103F20009847BDE80840FEF789BD00BF7C460020E9
:103F30004FF0B04310B5D3F8884004F47872C3F85A
:103F40008820A30604D5124A936A0BB1D06A984719
:103F5000600604D50E4A136B0BB1506B98472106CF
:103F600004D50B4A936B0BB1D06B9847E20504D58F
:103F7000074A136C0BB1506C9847A30504D5044A4B
:103F8000936C0BB1D06C9847BDE81040FEF756BD5E
:103F90007C4600204FF0B04310B5D3F8884004F4BD
:103FA0007C42C3F88820620504D5164A136D0BB114
:103FB000506D9847230504D5124A936D0BB1D06D0F
:103FC0009847E00404D50F4A136E0BB1506E984722
:103FD000A10404D50B4A936E0BB1D06E98476204CE
:103FE00004D5084A136F0BB1506F9847230404D5CA
:103FF000044A936F0BB1D06F9847BDE81040FEF7AD
:104000001DBD00BF7C46002008B50348FDF700F940
:10401000BDE80840FEF712BDCC23002008B5FFF72D
:10402000ABFDBDE80840FEF709BD0000062108B55C
:104030000846FFF7BBFA06210720FFF7B7FA06216B
:104040000820FFF7B3FA06210920FFF7AFFA06218F
:104050000A20FFF7ABFA06211720FFF7A7FA06217F
:104060002820FFF7A3FA09217A20FFF79FFA0721FA
:104070003220FFF79BFA0C215220BDE80840FFF7E1
:1040800095BA000008B5FFF78DFD00F00DF8FDF7BB
:10409000D1FAFDF7A9FCFDF77BFBFFF741FDBDE879
:1040A0000840FFF763BC00000023054A19460133AE
:1040B000102BC2E9001102F10802F8D1704700BFCD
:1040C0007C46002010B501390244904201D1002005
:1040D00005E0037811F8014FA34201D0181B10BD71
:1040E0000130F2E7034611F8012B03F8012B002AF7
:1040F000F9D1704753544D333248373F3F3F005357
:10410000544D3332483734332F37353300000000F5
:10411000F0290020CC2300200096000000000000C1
:10412000000000000000000000000000000000008F
:1041300000000000FD150008E9150008251600081C
:10414000111600081D16000809160008F5150008CC
:10415000E115000831160008000000000D170008E6
:10416000F916000835170008211700082D17000858
:104170001917000805170008F11600084117000874
:104180000000000001000000000000006D61696E89
:104190000000000069646C650000000094410008A4
:1041A00078280020F0290020010000008520000868
:1041B00000000000486F6C7962726F0025424F4129
:1041C0005244252D424C002553455249414C25006F
:1041D00002000000000000002D1900089D190008D1
:1041E0004000400098420020A84200200200000049
:1041F000000000000300000000000000E5190008B6
:104200000000000010000000B84200200000000084
:1042100001000000000000002C4500200101020008
:1042200075240008852300082124000805240008BF
:10423000430000003842000809024300020100C0A8
:1042400032090400000102020100052400100105EA
:10425000240100010424020205240600010705824E
:10426000030800FF09040100020A0000000705011D
:10427000024000000705810240000000120000001B
:1042800084420008120110010200004062314B001C
:1042900000020102030100000403090425424F410A
:1042A00052442500447572616E64616C0030313295
:1042B00033343536373839414243444546000000EF
:1042C00000000000391B0008F11D00089D1E0008B9
:1042D00040004000644600206446002001000000C9
:1042E000744600208000000040010000080000002B
:1042F0000001000000040000080000000000802A07
:1043000000000000AAAAAAAA00000024FFFF0000E3
:104310000000000000A00A000400000000000000EF
:10432000AAAAAAAA00000000FDFF000000000000E9
:10433000000000000050000000000000AAAAAAAA85
:10434000000000003FFF000000000000000000002F
:104350000000000000000000AAAAAAAA00000000B5
:10436000FFFF000000000000000000000004020049
:1043700000000000AAAAAAAA00080100DFFF0000AE
:1043800000000000070000005025100000000000A1
:104390000AA2AAAA50151000FFFF000000000007A3
:1043A000000000000000100000000000AAAAAAAA55
:1043B00000001000FFFF00000000000000000000EF
:1043C0000004000000000000AAAAAAAA000400003D
:1043D000FFFF00000000000000000000005111007D
:1043E00000000000AAAAAAAA00511100FFFF0000C5
:1043F00000000000000000000000000000000000BD
:10440000AAAAAAAA00000000FFFF00000000000006
:10441000000000000000000000000000AAAAAAAAF4
:1044200000000000FFFF000000000000000000008E
:104430008B0000000000000000001E0000000000D3
:10444000FF00000000000000F44000083F000000F2
:1044500050040000FF4000083F00000000960000EC
:1044600000000800960000000008000004000000A2
:10447000984200080000000000000000000000005A
:0C44800000000000000000000000000030
:00000001FF
